:1000000029C1000043C1000041C100003FC1000000
:100010003DC100003BC1000039C1000037C10000F4
:1000200035C1000033C1000031C100000C9425101F
:100030002DC100002BC1000029C10000F2C7000043
:1000400025C1000023C1000021C10000ABC1000098
:100050001DC100001BC1000019C1000017C1000034
:1000600015C1000013C1000011C100000FC1000044
:100070000DC1000012011001FF000010EB0304216C
:10008000000201020301090220000101008032097F
:1000900004000002FF0000000705820240000A077A
:1000A00005020240000A0403090418034400650025
:1000B00061006E002000430061006D006500720069
:1000C000610000002E034C00550046004100200056
:1000D00041005600520049005300500020004D00DE
:1000E0006B0049004900200043006C006F006E0067
:1000F000650000001C03300030003000300041007B
:100100003000300031003200380032003500350058
:1001100000000400040004000500050006000600BD
:100120000600070007000700080009000900090091
:100130000A000A000B000C000C000D000E000F005E
:100140000F0010001100120013001400150016001B
:100150001700180019001B001C001E001F002100C2
:1001600022002400260028002A002C002E00310046
:100170003300360039003B003E0041004500480096
:100180004C004F00540058005C00610065006A009C
:10019000700075007B00810088008E0096009D0035
:1001A000A500AD00B500BE00C800D200DC00E7002D
:1001B000F200FE000A011801250134014301530138
:1001C0006401760188019B01AF01C501DB01F301E8
:1001D0000B02250240025C027A029902BA02DC029A
:1001E000000326034E037703A303D1030104320463
:1001F00067049F04DA04150555059705E1052806EF
:100200007606C7061F077A07D7073308A308090928
:100210007A09F609700AF70A7C0B0D0CAD0C480D33
:10022000F20D920E410F0110D510971198128713FD
:1002300078147B158C16A417D018091A501BA21C11
:100240000B1E8C1F1921AF226F243726404000411E
:100250000142430011241FBECFEFD2E0DEBFCDBF6D
:1002600011E0A0E0B1E0E4E3F6E202C005900D92F7
:10027000A234B107D9F711E0A2E4B1E001C01D92A8
:10028000A535B107E1F74CD00C941813B9CE8BB15A
:1002900080658BB908958BB18F7A80618BB9089591
:1002A0008EB3843081F4B2D182E08093E9008091F2
:1002B000E80082FF08C08BB180658BB986D08BB116
:1002C0008F7A80648BB9089582E060E842E30E94EF
:1002D000800F80FD02C090E101C090E48BB18F7A65
:1002E000982B9BB9089584B7877F84BF88E10FB6A8
:1002F000F89480936000109260000FBE80E090E060
:1003000020E80FB6F89420936100809361000FBE3F
:100310008AB180658AB98BB18F7A8BB90C9416102B
:10032000E2DF6CD18BB18F7A80618BB9789489B11F
:100330008BB18BB9B5DF0E94EC12F9CFDA019230A4
:1003400049F0933061F0913029F5E4E7F0E022E1E3
:1003500030E024C0E6E8F0E020E230E01FC0813069
:1003600059F0813028F0823059F0833099F40CC074
:10037000E6EAF0E084910BC0EAEAF0E0849107C07D
:10038000E4ECF0E0849103C0E4EFF0E08491282FE6
:1003900030E004C0E0E0F0E020E030E0ED93FC93DA
:1003A000C901089578941F920F920FB60F921124ED
:1003B0008F938AB5882319F08AB581508ABD8F91B1
:1003C0000F900FBE0F901F901895FF920F931F93E1
:1003D0001091F10084E68ABD85E085BD143109F4F1
:1003E000CBC0153110F51A3009F4ADC01B3068F4DC
:1003F000143038F4123008F054C0113009F0D4C071
:1004000033C0163009F0D0C078C0113109F4AFC044
:10041000123120F4103109F0C7C0A7C0123109F41D
:10042000AEC0133109F0C0C0A4C0193109F4ACC08A
:100430001A3168F4163109F49FC0163108F499C0D6
:10044000173109F4A1C0183109F0AEC09AC01D31AE
:1004500009F49DC01D3108F494C0103509F49BC007
:10046000113509F0A1C095C08091E8008B77809389
:10047000E80082E08093E9008091EC008160809345
:10048000EC001093F1001092F1008AE08093F100EB
:1004900080E091E06AE070E040E050E00E94B1123C
:1004A00099C00091F100123011F0FF2402C0F090C9
:1004B000F1008091E8008B778093E80082E08093E0
:1004C000E9008091EC0081608093EC001093F100D2
:1004D000802FB5D0123041F481FF0DC01092F10091
:1004E000802F6F2DB4D076C080FF05C01092F10030
:1004F000802F9DD06DC080EC6BC084E491E064E0FF
:1005000070E040E050E00E943B128091E8008B7761
:100510008093E80082E08093E9008091EC008160A4
:100520008093EC008091440190914501A091460197
:10053000B0914701B7FF03C081E08093430186E09B
:100540008093F1000FC08091E8008B778093E800E2
:1005500082E08093E9008091EC0081608093EC0060
:100560001093F1001092F10035C0BED438C088D489
:1005700036C0812FF2D233C0812F41D230C0F0D1AA
:100580002EC0812FE5D02BC0812F9CD028C04BD10D
:1005900026C07ED624C0ADD722C08091E8008B77DC
:1005A0008093E8000E94B20F8091F2008034A9F39A
:1005B0008091E8008B778093E80082E08093E900E7
:1005C0008091EC0081608093EC001093F10089EC45
:1005D0008093F1008091E8008E778093E80015BC4D
:1005E0000E94B20F82E08093E9008091EC008E7F40
:1005F0008093EC001F910F91FF9008958DE487BDCB
:1006000082E084BD80936E0035D037C50895982F61
:10061000EBE0F1E08081981741F081E0E632F807E5
:1006200011F03396F7CFE0E0F0E0CF010895EFDF6F
:10063000FC01009711F480E0089582810895E7DFBE
:10064000FC01009711F480E00895818108950F93D3
:100650001F93182F062FDBDFFC01009741F0028368
:100660001E3929F480E090E0602F0E9406131F914C
:100670000F9108950F931F938EE9C9DF8C0180E0DD
:1006800090E00E94FE12F80182831F910F9108955D
:10069000282F40ED57E003C0CA010197F1F722234C
:1006A00021F08AB521508823B9F70895982F8091B9
:1006B0002901882329F09EBD0DB407FEFDCF0895C2
:1006C000892F19C5DF92EF92FF920F931F93DF934B
:1006D000CF9300D000D0CDB7DEB7D82E8E010F5FFC
:1006E0001F4FC80164E070E040E050E00E947612C5
:1006F0008091E8008B778093E80082E08093E900A6
:100700008091EC0081608093EC0085E0E82EF12C74
:10071000EC0EFD1EF80181918F01C8DF0E151F053B
:10072000C9F7D092F1001092F1001092F10080917F
:10073000E8008E778093E8000F900F900F900F9055
:10074000CF91DF911F910F91FF90EF90DF9008956F
:10075000BF92CF92DF92EF92FF920F931F93DF939E
:10076000CF93CDB7DEB729970FB6F894DEBF0FBE93
:10077000CDBFB82ECE01059665E070E040E050E0B8
:100780000E9476128091E8008B778093E80082E0E7
:100790008093E9008091EC0081608093EC008E01F1
:1007A0000A5F1F4F7E010894E11CF11C9AE0C92EDC
:1007B000D12CCC0EDD1EF801908180912901882377
:1007C00031F09EBD0DB407FEFDCF8EB502C0892F5E
:1007D00092D4F70181937F010F5F1F4F0C151D0508
:1007E00051F7B092F1001092F1008D81FE01E80FF7
:1007F000F11D80818093F1001092F1008091E8005A
:100800008E778093E80029960FB6F894DEBF0FBE6E
:10081000CDBFCF91DF911F910F91FF90EF90DF90AF
:10082000CF90BF900895EF92FF920F931F93DF93A5
:10083000CF93CDB7DEB7C250D1400FB6F894DEBF2C
:100840000FBECDBFCE01019663E070E040E050E006
:100850000E94761234E0E32EF12CEC0EFD1E69812D
:10086000C70170E040E050E00E9476128091E800FD
:100870008B778093E80082E08093E9008091EC0020
:1008800081608093EC008DE18093F1001092F10083
:1008900000E00BC08981081728F4F701E00FF11D73
:1008A000808101C080E002DF0F5F8B81081790F329
:1008B00010E024E0E22EF12CEC0EFD1E2CC089810C
:1008C00090912901081778F4F701E00FF11D80815C
:1008D000992331F08EBD0DB407FEFDCF8EB501C05A
:1008E0000AD40F5F0AC0992331F01EBC0DB407FE75
:1008F000FDCF8EB502C080E0FED38093F1008091E1
:10090000E80085FD07C08091E8008E778093E800BD
:100910000E94B20F1F5F8A81181788F21092F100AF
:100920009091E8008091E8008E778093E80095FD33
:1009300009C00E94B20F8091E8008E778093E80092
:100940000E94B20FCE5FDE4F0FB6F894DEBF0FBE2F
:10095000CDBFCF91DF911F910F91FF90EF90089540
:10096000EF92FF920F931F93DF93CF9300D000D0AD
:1009700000D0CDB7DEB7CE01019666E070E040E072
:1009800050E00E9476128091E8008B778093E80017
:1009900082E08093E9008091EC0081608093EC001C
:1009A0008E010D5F1F4F47E0E42EF12CEC0EFD1E73
:1009B000F80181918F017ADE0E151F05C9F78A8132
:1009C000882321F4898164DE90E002C0BFD3982F90
:1009D00082E18093F1009093F1008091E8008E779E
:1009E0008093E80026960FB6F894DEBF0FBECDBF09
:1009F000CF91DF911F910F91FF90EF900895DF92BB
:100A0000EF92FF920F931F93DF93CF9300D00F923B
:100A1000CDB7DEB7F82ECE01019663E070E040E07E
:100A200050E00E94761299818A8189839A8380910D
:100A3000E8008B778093E80082E08093E900809162
:100A4000EC0081608093EC00F092F1001092F100D4
:100A500000E010E068E0D62EEE24E39459C08091C7
:100A60004301882319F090D3109243018B811EDE3D
:100A70008091440190914501A0914601B0914701B8
:100A8000892F9A2FAB2FBB2711DE809144010EDEF8
:100A900080912901882331F01EBC0DB407FEFDCFE3
:100AA0008EB502C080E027D38093F1008091E800EA
:100AB00085FD07C08091E8008E778093E8000E9452
:100AC000B20F24E1F21619F48B818D258B8300FD82
:100AD00003C086E1F816D1F480914401909145015C
:100AE000A0914601B09147010196A11DB11D8093CF
:100AF000440190934501A0934601B093470126E13C
:100B0000F21621F0892B11F4E09243010F5F1F4F81
:100B100089819A810817190708F4A1CF1092F10072
:100B20009091E8008091E8008E778093E80095FD31
:100B300009C00E94B20F8091E8008E778093E80090
:100B40000E94B20F0F900F900F90CF91DF911F91E5
:100B50000F91FF90EF90DF9008954F925F926F9208
:100B60007F928F929F92AF92BF92CF92DF92EF923D
:100B7000FF920F931F93DF93CF93CDB7DEB7C9508A
:100B8000D1400FB6F894DEBF0FBECDBFB82ECE0158
:100B9000019669E070E040E050E00E9476126A81C0
:100BA000798131E06130730798F08091E8008B77AC
:100BB0008093E80082E08093E9008091EC008160FE
:100BC0008093EC00B092F10080EC8093F1003BC187
:100BD0007A836983CE010A9640E050E00E94761243
:100BE0008091E8008B778093E80082E08093E900B1
:100BF0008091EC0081608093EC0083E1B81611F4E1
:100C0000588401C059848B8180FD0FC066247724ED
:100C10000AE0C02ED12CCC0EDD1EEE24FF2420E0F5
:100C200018E0412EAA24A39404C17090440180903E
:100C3000450180914301882319F0A6D21092430107
:100C4000CC24DD24BAE0EB2EF12CEC0EFD1E00E0EE
:100C500010E0A8E06A2E4DC0992493949022F701E9
:100C6000A0808D8123DD8091440190914501A09168
:100C70004601B0914701892F9A2FAB2FBB2716DD74
:100C80008091440113DD8A2D11DDF3E1BF1619F4C3
:100C90008D8186258D83C114D10471F4A51461F072
:100CA000992031F033E1B31619F48F8188608F8376
:100CB000C0904401D0904501992019F485E1B816FF
:100CC00099F48091440190914501A0914601B09121
:100CD00047010196A11DB11D8093440190934501E8
:100CE000A0934601B09347010894E11CF11C0F5FEB
:100CF0001F4F89819A810817190708F4ADCF8B819E
:100D000087FD02C020E09BC08E81D0DC882DCEDC28
:100D1000872DCCDC80E0CADCC114D10431F48B8196
:100D200085FF03C08F7D80618B838B81B601452D4C
:100D30002C810F8132D2282FE3E1BE1609F07FC04B
:100D40008091440190914501892B09F078C081E0A0
:100D50008093430174C0E1E08E2E912C8E209F2061
:100D6000F601008180914301882319F00DD2109281
:100D700043018D819BDC8091440190914501A091BC
:100D80004601B0914701892F9A2FAB2FBB278EDCEC
:100D9000809144018BDC802F89DCF3E1BF1619F4CC
:100DA0008D8184258D831B81051571F0811491043B
:100DB00031F033E1B31619F48F8188608F8360902E
:100DC00044017090450106C013FD04C0812F8B7F44
:100DD00082608B838B81B301452D2C810F81DDD106
:100DE000282F882361F5892819F485E1B816D1F4F4
:100DF0008091440190914501A0914601B091470135
:100E00000196A11DB11D8093440190934501A093CB
:100E10004601B0934701E5E1BE1621F0892B11F49C
:100E2000A09243010894C11CD11C1B830894E11CAF
:100E3000F11C89819A81E816F90608F48CCFB092EA
:100E4000F1002093F1008091E8008E778093E80014
:100E5000C75FDE4F0FB6F894DEBF0FBECDBFCF9198
:100E6000DF911F910F91FF90EF90DF90CF90BF9097
:100E7000AF909F908F907F906F905F904F9008956C
:100E80000F931F93DF93CF9300D0CDB7DEB7CE0182
:100E9000019662E070E040E050E00E94761208EEB9
:100EA00010E0F80180818B77808382E08093E900F5
:100EB000ECEEF0E08081816080838981E9DB80E075
:100EC000AFD1EDD08A81E4DBE1EFF0E081E1808316
:100ED0001082F80180818E7780830F900F90CF91E0
:100EE000DF911F910F9108956F927F928F929F9241
:100EF000AF92BF92DF92EF92FF920F931F93DF9317
:100F0000CF93CDB7DEB72F970FB6F894DEBF0FBEE5
:100F1000CDBFCE0105966BE070E040E050E00E944E
:100F200076128091E8008B778093E80082E08093CE
:100F3000E9008091EC0081608093EC001092440104
:100F40001092450110924601109247018F81A0DB5B
:100F500073D120ECD22E9CE0692E712C6C0E7D1E7C
:100F60004E010894811C911C80E1A82EB12CAC0E7E
:100F7000BD1E30C09150988781E052D18E8188DBB0
:100F800083017401898584DBF801908180912901B6
:100F9000882331F09EBD0DB407FEFDCF8EB502C093
:100FA000892FA9D0F70181937F010F5F1F4F0A1589
:100FB0001B0541F78B85882361F0FE01E80FF11DC9
:100FC00090818A85981729F080E02AD18E8160DB94
:100FD00001C0DD249885992331F0F0ECDF1619F477
:100FE0008AB5882339F680E18093F100D092F10030
:100FF0008091E8008E778093E8002F960FB6F894E2
:10100000DEBF0FBECDBFCF91DF911F910F91FF903B
:10101000EF90DF90BF90AF909F908F907F906F90F8
:1010200008951F920F920FB60F9211248F93199962
:1010300008C08091490187FF02C02A9A17C02A98E8
:1010400015C080914901880F809349018091480122
:101050008150809348018F5F11F4109281001B9B97
:1010600005C080914901816080934901199A8F914F
:101070000F900FBE0F901F9018953E9A10926F0020
:1010800010928500109284001092890010928800BE
:1010900080E48093800089E08093810008958091AE
:1010A0002901882349F084B1897F84B985B1867F7D
:1010B00085B91CBC1DBC089584B1897F84B985B1F4
:1010C000867F85B9DACF92E090936F001092850009
:1010D00010928400E82FF0E0EE0FFF1FEC5FFE4F50
:1010E000859194919093890080938800109280005C
:1010F0001092810008958093490185E08093480112
:101100008091490180FF02C02A9A01C02A9810925A
:101110008500109284008AE08093810080914801CC
:10112000882319F08AB58823C9F71092810080912D
:1011300049010895982F80912901882329F09EBDA7
:101140000DB407FEFDCF0895892FD5CF80EFF2DFD4
:1011500080E0F0DF80E0EEDF80912901882331F02C
:101160001EBC0DB407FEFDCF8EB502C080E0C3DF0C
:1011700080FF03C08AB5882349F78AB5882311F414
:1011800081E8089580E008958DE4D4DF80E0D2DF27
:1011900080914601CFDF80E0CDCFEF92FF920F9399
:1011A0001F937B01142F90E08E778830910581F199
:1011B0008930910534F48230910559F0049751F546
:1011C0000BC08032910541F08034910509F14097C0
:1011D00009F5822F5DDA1EC0802FACDF8F2DAADFCC
:1011E0008E2DA8DF80912901882331F01EBC0DB41B
:1011F00007FEFDCF8EB502C080E07DDF811719F4B8
:101200008AB5882349F78AB5882321F480E803C08A
:101210009DDF01C080E01F910F91FF90EF90089536
:10122000882339F0249A8EE902DA882319F42C9A5B
:10123000089524982C98089588E9F9D9E82F8730E3
:10124000E8F481E080932901F0E0E45BFD4FE49154
:101250009E2F906184B1866084B984B1867F84B901
:1012600085B1896085B9E065ECBD96FF03C08DB599
:10127000816002C08DB58E7F8DBD089510922901C9
:1012800084B1866084B985B1896085B98E2F1BCF02
:10129000DF93CF930F92CDB7DEB7CE01019661E019
:1012A00070E040E050E00E9476128091E8008B7779
:1012B0008093E80082E08093E9008091EC008160F7
:1012C0008093EC0099819093420181E58093F10035
:1012D000913011F480EC01C080E08093F1008091A6
:1012E000E8008E778093E8000F90CF91DF9108950A
:1012F000AF92BF92CF92DF92EF92FF920F931F9324
:10130000DF93CF93CDB7DEB7C850D1400FB6F89476
:10131000DEBF0FBECDBFCE01019668E070E040E0B9
:1013200050E00E9476123B812C819D818E818B83BF
:101330009C832D833E837F8168856F8378878E01B0
:10134000075F1F4FC80140E050E00E947612809175
:10135000E8008B778093E80082E08093E900809139
:10136000EC0081608093EC0080914201882379F544
:1013700089818330A9F0843028F4813069F082308B
:10138000A9F40CC0853031F0853008F44AC08630AD
:1013900069F40AC088E046C044E209C04CE207C0D4
:1013A00045E383E366E305C04AE101C04EE283E220
:1013B00066E2EB80FC800D811E81AF80B8842A81BB
:1013C00099E0C92ED12CCC0EDD1EDFD206C04F8194
:1013D00058858B819C81B801E6D4882311F090E078
:1013E00001C093E080E58093F10084E08093F100F8
:1013F0009093F1008091E8008E778093E800C85FB9
:10140000DE4F0FB6F894DEBF0FBECDBFCF91DF9198
:101410001F910F91FF90EF90DF90CF90BF90AF9012
:1014200008958CE44B815C816D817E81298514D384
:10143000D4CFDF93CF93CDB7DEB7C750D1400FB62F
:10144000F894DEBF0FBECDBFCE01019667E070E01D
:1014500040E050E00E9476129A81EB817C816D81A0
:101460006A837B83EC839D833E812F812E833F8320
:101470008091E8008B778093E80082E08093E90018
:101480008091EC0081608093EC0080914201AE017C
:10149000485F5F4F882319F48E2F00D304C0CB011F
:1014A000BA01A901B8D4882311F493E001C090E0F7
:1014B00080E58093F10085E08093F1009093F10046
:1014C000992341F46E817F81CE01089640E050E07F
:1014D0000E94B1128091E8008E778093E800C95F86
:1014E000DE4F0FB6F894DEBF0FBECDBFCF91DF91B8
:1014F0000895DF93CF93CDB7DEB729970FB6F89451
:10150000DEBF0FBECDBF9091F100943009F4ADC0A5
:10151000953048F49230A1F1933008F04DC09130ED
:1015200009F036C10AC0963009F4A3C0963008F419
:101530009EC0973009F02CC1DEC08091E8008B7707
:101540008093E80082E08093E9008091EC00816064
:101550008093EC0080914201882311F496D305C05A
:10156000823011F090E002C091D4982F80E58093F2
:10157000F10081E08093F10089278093F10003C19D
:101580008091E8008B778093E8009093E900809148
:10159000EC0081608093EC0080914201882311F47B
:1015A0006AD301C06DD480E58093F10082E080931E
:1015B000F1001092F100E7C0CE01059665E070E001
:1015C00040E050E093D7588549857E816F814E83F6
:1015D0005F83688779878091E8008B778093E80044
:1015E00082E08093E9008091EC0081608093EC00C0
:1015F000809142019D81882339F59430C1F0953066
:1016000038F4923071F0933080F49130D1F40BC003
:10161000963089F0963068F0973079F0983089F4F8
:101620000EC080E20FC080E40DC088E60BC080E3EE
:1016300009C082E207C08AE205C082E303C088E1F4
:1016400001C080E06FD207C0913011F084E101C089
:1016500080E1BA018DD3882311F090E001C093E0BE
:1016600080E58093F10083E08AC042DE91C0E1DE34
:101670008FC0CE01059661E070E040E050E036D7C3
:101680008091E8008B778093E80082E08093E90006
:101690008091EC0081608093EC008091420188236E
:1016A00011F091E013C08D81813021F0823021F45E
:1016B00089E303C088E301C088E7BE016F5F7F4F05
:1016C0009ED2882311F493E001C090E080E58093DE
:1016D000F10086E08093F1009093F100992309F0E6
:1016E00052C089819A81AB81BC819D0144275527D5
:1016F0002093F10044C08091F1008230E1F083300A
:1017000018F4813029F406C08330F1F0843009F1F7
:1017100091E024C03091F1002091F1009091F1000E
:101720008091F10080932A0190932B0120932C014A
:1017300030932D0112C09091F1008091F1008093BF
:101740002E0190932F0109C08091F1008093300108
:1017500004C08091F1008093310190E08091E80015
:101760008B778093E80082E08093E9008091EC0021
:1017700081608093EC0080E58093F10087E08093A6
:10178000F1009093F1008091E8008E778093E8005B
:1017900029960FB6F894DEBF0FBECDBFCF91DF9173
:1017A00008954D99FECF4D9BFECF5B9A539A809141
:1017B000C9008F7E8093C9008091C90088608093A2
:1017C000C90081E080934A01089580914A018823ED
:1017D00009F4E7DF80E04D99FECF4D9BFECF8F5F90
:1017E0008C30C9F7089510924A01249A2C9882E00F
:1017F0008A95F1F78AB188628AB952988FE090E0B1
:101800009093CD008093CC0088E08093C9008FE650
:101810008093CA00DADFD9CF10924A018AB1886278
:101820008AB952985B9A82E08A95F1F78FE090E04E
:101830009093CD008093CC0088E08093C9008FE620
:101840008093CA00C2DFC1CF1F93182F80914A0135
:10185000882309F4A6DF8091C80085FFFCCF809122
:10186000C80080648093C8001093CE001F91089533
:101870008091C80086FFFCCF8091C800806480936F
:10188000C8008091C900877F8093C9008091C900FA
:1018900080618093C90053985B9810924A01089523
:1018A00080914A01882309F0E3DF8091C80087FD19
:1018B00003C08AB58823C9F78091CE000895D8DF88
:1018C000E8ECF0E08081806C80831092C900109277
:1018D000CA008AB1877D8AB98BB1837D8BB9249880
:1018E0002C980895C5DF80EC8093C8001092C90041
:1018F0001092CA008AB1877D8AB98BB1837D8BB97A
:1019000008950F931F93DF93CF9300D000D0CDB7EE
:10191000DEB769837A838B839C838E010F5F1F4FB1
:10192000862F92DFF80181818FDFF80182818CDFC1
:10193000F801838189DF0F900F900F900F90CF9166
:10194000DF911F910F91089590E0A0E0B0E0209109
:101950002A0130912B0140912C0150912D01822BB5
:10196000932BA42BB52BBC01CD01CBCF8BE66CDF29
:101970008FE0EADF80E268DF93DF982F8AB5882363
:1019800019F097FDF7CF81E008957F928F929F9293
:10199000AF92BF92CF92DF92EF92FF920F931F937D
:1019A000CF93DF93882E962E742EE601D22E20FF41
:1019B00010C0DCDF882309F440C08CE445DF8AE0F6
:1019C000C3DF892D41DF8CE43FDF8BE0BDDF81E0A9
:1019D0003BDFA114B104E9F0C9DF882371F18CE485
:1019E00033DF8AE0B1DF882D2FDF8BE62DDFC801E2
:1019F000B70187DF80EA28DF8A2D815025DF84E662
:101A000023DF899121DF0894A108B108A114B10452
:101A1000C1F7D1FE10C0AADF882379F08CE414DF6F
:101A20008AE092DF872D10DF8CE40EDFC801B7015A
:101A300068DF80E009DF81E001C080E0DF91CF91C5
:101A40001F910F91FF90EF90DF90CF90BF90AF90DC
:101A50009F908F907F900895CF92DF92EF92FF92A8
:101A60000F931F93D82E7A018B01C22E7FDF88231C
:101A700071F08CE4E9DE8AE067DF8D2DE5DE8CE431
:101A8000E3DEC801B7013DDF8C2DDEDE81E01F9172
:101A90000F91FF90EF90DF90CF900895CF92DF925B
:101AA000EF92FF920F931F93CF93DF937B018C01F3
:101AB0006A01E9015BDF882309F18CE4C5DE8AE075
:101AC00043DF83E4C1DE8BE6BFDEC801B70119DF67
:101AD00080EABADE9E012150822FB6DE84E2B4DEB7
:101AE00004C0DEDEF60181936F01209721F08AB5F4
:101AF00021978823B1F78AB5811181E0DF91CF91D9
:101B00001F910F91FF90EF90DF90CF90089580E8A4
:101B10009BDEC6DE982F8AB5882319F091FFF7CF98
:101B200081E00895CF92DF92EF92FF921F93182FDA
:101B30006A017B011BDF882309F45AC0103431F499
:101B40008CE482DE8AE000DF80E439C0103309F0E3
:101B50003DC08CE479DE8AE0F7DE86E375DE8CE456
:101B600073DE8BE0F1DE81E06FDE00DF882309F4B5
:101B70003FC08CE469DE8AE0E7DE83E365DE8BE666
:101B800063DEC701B601BDDE80EA5EDE80912E0114
:101B900081505ADE84E658DE10E003C080E054DE57
:101BA0001F5F212F30E080912E0190912F01281787
:101BB0003907A0F38CE448DE8AE0C6DE80E344DE29
:101BC0008CE442DE8BE0C0DE81E00CC08CE43CDEC5
:101BD0008AE0BADE812F38DE8CE436DEC701B6013A
:101BE00090DE80E031DE93DF882319F081E001C0D0
:101BF00080E01F91FF90EF90DF90CF900895EF92DB
:101C0000FF920F931F93082FF62EE72EAFDE882347
:101C100061F18CE419DE8AE097DE802F15DE8CE41A
:101C200013DE8BE091DE81E00FDE71DF8823E9F0C7
:101C30009DDE8823D1F08BE607DE84E085DE80EA36
:101C400003DE82E001DE84E2FFDD0F2D1E2D28DEA3
:101C5000F801808325DEF801818322DEF80182838A
:101C60008AB5882319F081E001C080E01F910F91AF
:101C7000FF90EF9008954BDF81ECE6DD80E0E4DD3E
:101C800081ECE2DD80E0E0DD2DCEEF92FF920F935C
:101C90001F93DF93CF93CDB7DEB728970FB6F89495
:101CA000DEBF0FBECDBFB8DD81ECCEDD89E5CCDD7A
:101CB00082ECCADD87E0C8DD80EEC6DD8E01085FFC
:101CC0001F4F7E010894E11CF11CD701E2E3F1E013
:101CD00088E001900D928150E1F7F8018081B4DD38
:101CE000015010400C171D0781F711DF28960FB621
:101CF000F894DEBF0FBECDBFCF91DF911F910F9142
:101D0000FF90EF900895282F8F70806930E0207346
:101D10003070220F331F822B97CDDF93CF9300D0EB
:101D2000CDB7DEB79A83898388E68EDD89818CDD25
:101D300089E68ADDFE013196818186DD0F900F9064
:101D4000CF91DF91089520913101822F8F708061B2
:101D500030E020733070220F331F822B75DDA0DD41
:101D6000982F8AB5882319F097FDEDCF81E008956B
:101D70001F93CF93DF93182FEB01E5DF882379F0D2
:101D800080913001C0DF812F5FDDCE018160C5DF32
:101D900080E65ADD80E058DDD6DF811181E0DF91F9
:101DA000CF911F910895EF92FF920F931F93CF93BE
:101DB000DF937C018B01EA01C6DF882321F1C0FF9C
:101DC00006C0F801EC0FFD1F8FEF808321968091F4
:101DD000300199DF8DE138DDC7019FDF10C0B3DF2F
:101DE000882389F084E630DDF80180812DDD84E6EA
:101DF0002BDDF80181810E5F1F4F26DD2297209792
:101E000071F781E001C080E0DF91CF911F910F91C8
:101E1000FF90EF900895EF92FF920F931F93CF934F
:101E2000DF938C017B01EA018EDF8823B9F080917A
:101E3000300169DF80E008DDC8016FDF06C084E2A1
:101E400003DD2EDDF70181937F01209721F08AB514
:101E500021978823A1F78AB5811181E0DF91CF9185
:101E60001F910F91FF90EF90089580E8EDDC18DD51
:101E7000982F8AB5882319F091FFF7CF81E0089554
:101E8000F4DF80ECE1DC80E0DFDC19CDEF92FF9243
:101E90000F931F93DF93CF93CDB7DEB728970FB67D
:101EA000F894DEBF0FBECDBF9EDC82ECCDDC87E0B8
:101EB000CBDC80EEC9DC8E01085F1F4F7E010894E9
:101EC000E11CF11CD701EAE3F1E088E001900D92FA
:101ED0008150E1F7F8018081B7DC015010400C1708
:101EE0001D0781F7C2DF28960FB6F894DEBF0FBE3C
:101EF000CDBFCF91DF911F910F91FF90EF9008958B
:101F00008093E9008091EB0081608093EB00109258
:101F1000ED006093EC004093ED008091EE00881F8F
:101F20008827881F089580914D0188238CF403C071
:101F30008EB38823B1F08091E80082FFF9CF8091C1
:101F4000E8008B778093E80008958EB3882349F0EA
:101F50008091E80080FFF9CF8091E8008E77809330
:101F6000E80008954091E4005091E50024E6809156
:101F7000EC0080FF05C08091E80080FF05C021C013
:101F80008091E80082FD1DC08EB3882311F482E0A9
:101F90000895853011F483E008958091EB0085FF6A
:101FA00002C081E008958091E4009091E5008417DB
:101FB0009507E9F2222311F484E008952150AC0141
:101FC000D6CF80E008953BD03DD08091D800982FA7
:101FD0009F779093D80080688093D80019BC89B50A
:101FE000826089BD09B400FEFDCF8091D8008F7D4D
:101FF0008093D8001EBA10924B0180E060E042E16D
:102000007FDF8091E1008E7F8093E1008091E2008C
:1020100081608093E2008091E20088608093E2001A
:102020008091E0008E7F8093E0000895E3E6F0E089
:1020300080818E7F808381E080934C01C4CF109299
:10204000E20008951092E10008951F920F920FB6DA
:102050000F9211242F933F934F935F936F937F932E
:102060008F939F93AF93BF93EF93FF938091E10082
:1020700080FF1CC08091E20080FF18C08091E100C9
:102080008E7F8093E1008091E2008E7F8093E2005A
:102090008091E20080618093E2008091D8008062AC
:1020A0008093D80019BC1EBA0E944B018091E100B8
:1020B00084FF2DC08091E20084FF29C019BC89B53E
:1020C000826089BD09B400FEFDCF8091D8008F7D6C
:1020D0008093D8008091E1008F7E8093E100809111
:1020E000E2008F7E8093E2008091E2008160809325
:1020F000E20080914B01882331F48091E30087FD59
:1021000002C081E001C084E08EBB0E944701809143
:10211000E10083FF21C08091E20083FF1DC0809118
:10212000E100877F8093E10082E08EBB10924B013B
:102130008091E1008E7F8093E1008091E2008E7FAC
:102140008093E2008091E20080618093E20080E071
:1021500060E042E1D5DE31D18091E10082FF0AC02A
:102160008091E20082FF06C08091E1008B7F809326
:10217000E10023D1FF91EF91BF91AF919F918F919A
:102180007F916F915F914F913F912F910F900FBE73
:102190000F901F9018950F931F93DF93CF9300D04C
:1021A000CDB7DEB7EDE4F1E08091F100819381E0FD
:1021B000E535F807C9F701D18091E80083FFE8C051
:1021C00080914D0190914E01953009F46DC096308B
:1021D00040F4913081F1913070F0933009F0D8C023
:1021E0002AC0983009F4A6C0993009F4B5C09630D9
:1021F00009F0CEC07EC0803809F4CAC0823809F028
:10220000C7C08091510187708093E9008091EB00F5
:102210001092E9002091E800277F2093E80090E0E9
:1022200025E0969587952A95E1F781708093F100D6
:102230001092F1008AC0882319F0823009F0A8C0FA
:102240008F71823009F0A4C080914F01882331F54D
:1022500020915101277009F49BC02093E9008091DF
:10226000EB0080FF1BC0933021F48091EB00806273
:1022700013C08091EB0080618093EB0081E090E0DF
:1022800002C0880F991F2A95E2F78093EA00109206
:10229000EA008091EB0088608093EB001092E900E7
:1022A0008091E800877F54C0882309F071C01091A5
:1022B0004F011F770FB7F8948091E800877F8093D4
:1022C000E80031DE8091E80080FFFCCF112311F49B
:1022D00082E001C083E08EBB8091E3008078182B00
:1022E0001093E3008091E30080688093E3000FBFC8
:1022F0004FC08058823008F04BC080914F019091C0
:10230000500160915101AE014F5F5F4F0E949E01ED
:10231000BC01009709F43CC08091E800877F80935E
:10232000E80089819A814AD08091E8008B77809378
:10233000E8002EC0803861F58091E800877F8093A7
:10234000E80080914B018093F1008091E8008E7746
:102350008093E800E8DD1CC08823D1F490914F0100
:102360009230B0F48091E800877F8093E8009093EA
:102370004B01D9DD80914B01882331F48091E3003A
:1023800087FD02C081E001C084E08EBB0E94640131
:102390008091E80083FF0AC08091EB008062809307
:1023A000EB008091E800877F8093E8000F900F900A
:1023B000CF91DF911F910F91089508959C01409155
:1023C0005301509154014617570710F460E03EC086
:1023D0006115710511F0AB01F9CF8091E8008E779E
:1023E0008093E80040E050E0F1CF8EB3882309F4F9
:1023F0003EC0853009F43DC08091E80083FF02C0F3
:1024000081E008958091E80082FD2BC08091E80072
:1024100080FF1CC08091F20090E009C0F9012F5F9D
:102420003F4FE491E093F100415050400196411537
:10243000510519F08031910588F360E0409709F467
:1024400061E08091E8008E778093E80041155105A6
:1024500061F6662351F605C08EB3882341F08530BE
:1024600041F08091E80082FFF7CF80E0089582E09C
:10247000089583E00895DF92EF92FF920F931F93E8
:10248000CF93DF938C01EB017A016CDDD82E88238A
:1024900021F521970C0F1D1F21961DC08091E8008A
:1024A00085FD12C08091E8008B778093E800E114ED
:1024B000F10431F0F7010995813011F485E00EC087
:1024C00051DD882341F00AC08091F100F80180833A
:1024D000015010402197209709F78D2DDF91CF9162
:1024E0001F910F91FF90EF90DF900895DF92EF9290
:1024F000FF920F931F93CF93DF93182F092FEB01B8
:102500007A0130DDD82E882319F5812F902F9C0178
:1025100089011CC08091E80085FD12C08091E8000F
:102520008B778093E800E114F10431F0F70109950D
:10253000813011F485E00DC015DD882339F009C024
:102540008091F100F80181938F012197209711F775
:102550008D2DDF91CF911F910F91FF90EF90DF9024
:102560000895DF92EF92FF920F931F93CF93DF9323
:10257000182F092FEB017A01F5DCD82E882319F5E5
:10258000812F902F9C0189011CC08091E80085FD5E
:1025900012C08091E8008E778093E800E114F10486
:1025A00031F0F7010995813011F485E00DC0DADCD6
:1025B000882339F009C0F80181918F018093F100DF
:1025C0002197209711F78D2DDF91CF911F910F91BA
:1025D000FF90EF90DF9008951F938EB3882361F0F2
:1025E0001091E9001092E9008091E80083FF01C09A
:1025F000D2DD17701093E9001F910895F999FECF6D
:1026000092BD81BDF89A992780B50895262FF99932
:10261000FECF92BD81BDF89A019700B4021639F041
:102620001FBA20BD0FB6F894FA9AF99A0FBE089512
:04263000F894FFCF4C
:102634004156524953505F4D4B3200800100810195
:102644000090010091010192010D9401329803035D
:102654009E0201A10100A4020001C00100012000AA
:1026640033321289AB45CDD888FF1289AB45CDD81A
:0226740088FFDD
:00000001FF
